:020000040000FA
:06000000A3EF10F0120056
:06080000A3EF10F012004E
:06082A000200AC210000F9
:100830006000000020000000AA2100002B02000040
:0408400002000000B2
:0C0844005EEC09F0FB0EDBCFF3FFDB06DF
:10085000F35000090AE0ACEC09F0FA0E17EC0AF0CC
:10086000F3E1151CF1E1010E01D0000E8DEF09F04E
:100870005EEC09F03B0EE12402E3E168E652E16E32
:10088000010EDB6A020EDB6AF90EDBCFF6FFFA0E11
:10089000DBCFF7FFFB0EDBCFF8FF0800F550DF6E74
:1008A000DF5002E1B1EF08F0250EDF5C02E0A4EFBB
:1008B00008F0030EDB6A040EDB6A050EDB6A060E27
:1008C000DB6A070EDB6AC6EC08F02D0EDF5C0CE07D
:1008D0002B0EDF5C09E0200EDF5C06E0230EDF5C00
:1008E00003E0300EDF5C1AE1DF50300A14E0130A37
:1008F0000FE0030A0AE00B0A05E0060AE4E1030E32
:10090000DB80E1D7030EDB82DED7030EDB84DBD78F
:10091000030EDB86D8D7030EDB88D5D72A0EDF5C23
:100920001BE1C2EC08F010EC09F010E0030EDB80D4
:1009300008680968130EDBCF0DF0140EDBCF0EF044
:10094000D7EC0FF0040E06C0DBFF03D0130EF9EC5A
:1009500008F0C6EC08F00BD0090EDB6A67EC09F072
:1009600003E0DBEC09F0FAD7090EF9EC08F0030E0E
:10097000DBB0DB982E0EDF5C1BE1C6EC08F02A0E24
:10098000DF5C0BE1C2EC08F010EC09F003E1130EA0
:100990004BEC09F0C6EC08F00BD0090EDB6A67ECF3
:1009A00009F003E0DBEC09F0FAD7090E4BEC09F093
:1009B000680EDF5C07E1C6EC08F0680EDF5C1DE145
:1009C000030E18D0740EDF5C17E07A0EDF5C14E0C3
:1009D000480EDF5C06E0540EDF5C03E05A0EDF5C7D
:1009E00002E1020E07D06C0EDF5C03E06A0EDF5CF2
:1009F00004E1010E9EEC09F0C9DBDF506E0A01E153
:100A00007FD31E0A01E192D1200A01E18FD13F0A72
:100A100001E149D11A0A01E146D10D0A01E143D1B0
:100A2000200A01E140D13A0A01E13DD1200A01E169
:100A30003AD1260A01E135D10D0A01E132D11A0A73
:100A400001E1D9D0200A4AE0300A1FE0460A0EE050
:100A5000250A01E083D3D950F90FE96EFF0EDA20A1
:100A6000EA6E010EEE5E000EEE5AEE5AACEC09F0A4
:100A7000250EE66E95DB03E1151C01E169D3A8ECB8
:100A800009F001E26BD3DB2A69D3080EDB6A040E9E
:100A9000DB50010806E2040EDB0470EC09F0DB50C9
:100AA0008BDB080EDB5009E0030EDB50010B05E188
:100AB00072DB01E04DD3080EDB6A64DBEFCFDFFFB2
:100AC00020EC0AF003E1151C01E142D3A8EC09F087
:100AD00001E3DB2A60DB01E141D33AD3070EDB50AF
:100AE00002080FE1ECEC09F0030EB3EC09F00E0E76
:100AF000EECFDBFF0F0EEECFDBFF100EEECFDBFFF6
:100B000020D0F70EDBCF17F0F80EDBCF18F0020E77
:100B1000175E000E185AF70E17C0DBFFF80E18C04C
:100B2000DBFF17C0E9FF18C0EAFFA3EC09F0166A63
:100B30000E0E14C0DBFF0F0E15C0DBFF100E16C02B
:100B4000DBFF0E0EDBCFE6FF0F0EDBCFE6FF100E56
:100B5000DBCFE6FFB2EC0FF0E552E552E552130EA3
:100B600007C0DBFF140E08C0DBFF060EDB5005E0FC
:100B7000130EE7EC09F001E26ADB0BEC0AF002E28B
:100B8000130E37DBCEEC09F006E0040EE7EC09F0BB
:100B900002E2050E2EDB030EDBB005D0FCDA01E02D
:100BA000D7D2080EDB6A090EDB6A0E0EDBCFF6FF2A
:100BB0000F0EDBCFF7FF100EDBCFF8FF0800F5506C
:100BC000DF6EDF5014E011EC0AF011E220EC0AF0C5
:100BD00003E1151C01E1BCD2BBDB01E3DB2A090EFA
:100BE000DB2AD9500E0FE96E000ECBDBE7D7D3DA44
:100BF00001E1B4D2ADD2C6DA110EEECFDBFF120E98
:100C0000EDCFDBFF110EDBCFE6FF120EDBCFE6FFF1
:100C1000A4EC0FF0E552E552130EF3CFDBFF140EF8
:100C2000F4CFDBFF060EDB5004E0130ED0DB01E255
:100C30000EDB0BEC0AF002E2130EDBDAAFDB05E0B1
:100C4000040EC5DB02E2050ED4DA030EDBB005D0DC
:100C5000A2DA01E07DD2080EDB6A090EDB6A110E12
:100C6000DBCFE9FF120EDBCFEAFFEFCFDFFFDF5074
:100C700014E0D7DB12E2E4DB03E1151C01E168D2EA
:100C800067DB01E3DB2A090EDB2A110EDB2ADBCF4F
:100C9000E9FF120EE8E3DB2AE6D77DDA01E15ED256
:100CA00057D2030EDB8E070EDB0410E195DB040E3A
:100CB0005ADB0A0EEECFDBFF0B0EEECFDBFF0C0E86
:100CC000EECFDBFF0D0EEECFDBFF6CD0070EDB505F
:100CD00003082CE1030EDBAE0DD0B2DA020E76DA99
:100CE000EFCF14F0156A166A176A14AE39D015687A
:100CF000166835D0F70EDBCF15F0F80EDBCF16F007
:100D0000020E155E000E165AF70E15C0DBFFF80E28
:100D100016C0DBFF15C0E9FF16C0EAFFEFCF14F0E5
:100D20000A0E14C0DBFF0B0EDB6A38D0070EDB5057
:100D3000020809E1030EDBAE04D059DB16AE10D079
:100D40000ED055DB0DD0030EDBAE12D079DA020ED9
:100D50003DDAF9DA166A176A15AE02D01668176816
:100D6000E2DA0C0E16C0DBFF0D0E17C0DBFF1AD047
:100D7000F70EDBCF16F0F80EDBCF17F0020E165E83
:100D8000000E175AF70E16C0DBFFF80E17C0DBFF78
:100D900016C0E9FF17C0EAFFD6DAC5DA0C0EDB6A27
:100DA0000D0EDB6A060EDB5005E1010EF36E050E3B
:100DB000F3CFDBFF150EDB6A160EDB6AD950370F57
:100DC000146E000EDA20156E390E14C0DBFF3A0ED9
:100DD00015C0DBFF380EDB6A080EDB6A0A0EAEDADE
:100DE000DF50780A12E0200A10E0280A0CE0200AFE
:100DF0000AE03F0A06E00D0A02E0200A08E1020EBE
:100E000005D0080E03D0080EDF26100E97DA030E69
:100E1000DBBE02D0DB92DB94DB50800B24E08ADA6D
:100E2000D890030EEB50000A08E6000EEE5C000EB0
:100E3000EE58000EEE58000EEE5815E213DA0B686D
:100E40000C680D680E686CEC0FF00A0E02C0DBFF38
:100E50000B0E03C0DBFF0C0E04C0DBFF0D0E05C044
:100E6000DBFF2D0E08D0030EDBA202D02B0E03D029
:100E7000DBA408D0200EF36E170EF3CFDBFF150EA8
:100E8000DB2A02D0170EDB6A050EDB5003E1B7D96F
:100E900001E189D0940E146E210E156E000E166EAF
:100EA000070EDBCF17F0186A196A1A6A17C00BF021
:100EB00018C00CF019C00DF01AC00EF0D3D904EC14
:100EC00010F014500224F36E15500320F46E1650E7
:100ED0000420F86EF4CFF7FFF3CFF6FF0800090EF9
:100EE000F5CFDBFF580EDF5C0FE1610EF36E090EEC
:100EF0007BD90AE3200E146E090EDBCFE7FF1450F6
:100F0000E75E090EE7CFDBFF070EDBCF14F0156AB3
:100F1000166A176A0FDA14C00BF015C00CF016C071
:100F20000DF017C00EF0EECF06F0EECF07F0EECFCB
:100F300008F0EFCF09F004EC10F009C0EDFF08C095
:100F4000EDFF07C0EDFF06C0EFFF390EDBCFE9FF75
:100F5000DB063A0EDBCFEAFF01E2DB06090EDBCF50
:100F6000EFFF150EDB2A4BD995E1030EDBA61DD052
:100F70006F0EDF5C06E1C1D918E3150EDB285BDAE2
:100F800014D0780EDF5C09E0580EDF5C06E0620EDC
:100F9000DF5C03E0420EDF5C08E1020EF36E160E2A
:100FA000F3CFDBFF02D0150EDB6A030EDB50100B14
:100FB0000EE0040EDBCF14F0050EDB50D880145485
:100FC00006E2060EDB5003E1040EDB5034DA95D95D
:100FD0000AE2050EDBCFE7FF150EDB50E75E050EDC
:100FE000E7CFDBFF02D0050EDB6A040EDBCF14F087
:100FF000160E45D9D880145414E2160EDBCFE6FF46
:10100000150EDBCFE6FF040EDBCFE6FF050EDB504F
:10101000E552E75CE552D880E754E552D880E754C2
:101020005FD9030EDB50010B0BE1080EDB5008E02B
:10103000B2D801E08DD0080EDB50BED8080EDB6AB6
:10104000170EDB5007E088D9170EF1D903E1151C04
:1010500001E17ED0160EDB5016E07ED9300EE66E32
:101060009FD802E1151C74E077D9DFCFE6FF2AECA8
:101070000FF0E552E552E552F4CF15F00001F31CF4
:1010800002E1151C65E0050EDBCF14F0160EDB50F7
:10109000D880145409E2050EDBCFE7FF160EDB50B3
:1010A000E75E050EE7CFDBFF300EE66E050ECBD90F
:1010B0004FE1390EDB2ADBCFE9FF3A0E01E3DB2AF1
:1010C000DBCFEAFF090EEFCFDBFFDB500EE044D9A8
:1010D000090EADD902E1151C3BE0390EDB2ADBCF4E
:1010E000E9FF3A0EEDE3DB2AEBD755D831E1160ED6
:1010F000DBCFE6FF080EC3D8E552E7245DD82ED03B
:10110000070EDB50030A1CE0010A14E0030A07E0A3
:101110007BD9DBCFEEFF020EDBCFEDFF1FD0F5D882
:10112000196A17AE02D0186819682CD8BCD819C033
:10113000EEFF14D0EAD817BE186824D8B4D80ED061
:1011400063D9DBCFEFFF0AD07BD905E1151C03E1A2
:10115000F368F46810D0FCD801E3DB2A79D94DEFAD
:1011600004F0010EDBCF14F0020EDBCF15F014C03B
:10117000F3FF15C0F4FF3B0EE15C02E2E16AE552C9
:10118000E16ECBD029D9020EB3EF09F061D9080086
:10119000F550DF6E1200200EE66E080E23EF0AF007
:1011A0002AEC0FF0E552E552E552F3CF14F0F4CFFC
:1011B00015F00001F31C1200146E156AD950010FCE
:1011C0004DD91450EE261550ED221200185E000E77
:1011D000195AF70E18C0DBFFF80E19C0DBFF18C054
:1011E000E9FF19C0EAFF1200DBCFF4FFF350F45C13
:1011F0001200DB50E76E040EE7CFDBFF12000A0E91
:10120000DBCF14F00B0EDBCF15F00C0EDBCF16F09E
:101210000D0EDBCF17F0145015101610171012001A
:10122000130EEECFDBFF140EEDCFDBFF130EDBCF83
:1012300014F0140EDBCF15F00001800E151412000F
:10124000F70EDBCF18F0F80EDBCF19F01200050E09
:10125000DB50E66ED950130F01D9E552E750EE6E20
:10126000ED6A12000A0EDBCF06F00B0EDBCF07F0A3
:101270000C0EDBCF08F00D0EDBCF09F01200DBCF38
:10128000E6FF150EDBCFE6FF050EDB50E552E72447
:10129000E552E7241200DB50CED8010EF36E060EA5
:1012A000F3CFDBFF1200EE50EFCFEAFFE96E16C07E
:1012B000EEFF17C0EEFF18C0EEFF1200D9CFE6FF19
:1012C000DACFE6FFE1CFD9FFE2CFDAFF1200DFCFBE
:1012D000E6FFE66A71EC10F0E552E552F3501200B9
:1012E000E76E080EE7CFDBFF1200EECF14F0EECF73
:1012F00015F0EFCF16F0176A1200050EDBCF14F0D1
:10130000150EDB50D88014541200010EDBCF16F0FE
:10131000020EDBCF17F0186A1200E552E5CFDAFFB4
:10132000E7CFD9FF12000A0E14C0DBFF0B0E15C069
:10133000DBFF1200D9500A0F2EEF0AF0F36E070EF2
:10134000F3CFDBFF1200EECF14F0EFCF15F0120059
:10135000010EDB2A020E1200FC0EDBCFE6FFFD0EB3
:10136000DBCFE6FF1200145E000E155AF70E14C014
:10137000DBFFF80E15C0DBFF14C0E9FF15C0EAFF64
:101380001200DA20EA6EEF2AEECFF6FF000EEF220F
:10139000EECFF7FFEF22EECFF8FF1200040EDBCF07
:1013A000E6FF130EDB50E552E75C9ADFDB5004DF0B
:1013B000060EDB501200090EDB500A0DF350DF243D
:1013C000D00FE76E090EE7CFDBFFC6EF08F0DB506A
:1013D000F36E050EF4EF08F0F70EDBCF14F0F80E05
:1013E000DBCF15F01200DFCFE6FFD0EF08F028DFEB
:1013F000030EECDE75EF09F022EC04F0E552E55245
:10140000E552E55200091200BDDEEE50EFCFEAFFD3
:10141000E96E010E1200130EDB50F36E040EF4EFB2
:1014200008F0040EDB50F36E090EF4EF08F0DBCF8A
:10143000E6FFD0EF08F0E76E050EE7CFDBFF120006
:101440008BDFF3EF09F0DBCFE6FF86DFFCEF09F07F
:10145000D950F90FE96EFF0EC1EF09F0E96E000EE9
:06146000DA20EA6E120022
:0A146600D9CFE6FFE1CFD9FF040E55
:10147000E126DE6ADE6ADE6ADD6ADD52DD52FD0EDD
:10148000DBCF14F0FE0EDBCF15F0166A176A15AE2F
:1014900002D016681768D9CFE9FFDACFEAFF030E4A
:1014A000EB501718E8AE02D0173408D01450EE5C99
:1014B0001550EE581650EE581750EE580FE20C0E1D
:1014C000E66E83EC10F0E552D9CFE9FFDACFEAFF00
:1014D000EE2A000EEE22EE22EE22D1D7040EE15CBF
:1014E00002E2E16AE552E16EE552E7CFD9FF120070
:1014F0000F0EC16E070EB46E936A300E926E0F0E11
:10150000946EF19E1200D9CFE6FFE1CFD9FF020E13
:10151000E1268250020B01E0010E080DF3CF16F018
:101520008250010B040DF3CF15F08050200B01E029
:10153000010EE824146E8050100B01E0010E1424FB
:1015400015241624DE6EDD6ADECF14F0DDCF15F033
:1015500014C0F3FF15C0F4FF020EE15C03E200D0FB
:10156000E16AE552E16EE552E7CFD9FF12008092C1
:10157000320EE66EBFEC10F0E5528084320EE66E5D
:10158000BFEC10F0E5528094320EE66EBFEC10F026
:10159000E55212008082320EE66EBFEC10F0E5528A
:1015A0008084320EE66EBFEC10F0E5528094320E6D
:1015B000E66EBFEC10F0E5521200380E816ED7DFF8
:1015C000320EE66EE66A4FDFE552E552010E816E9D
:1015D000CEDF320EE66EE66A46DFE552E5520D0ECC
:1015E000816EC5DF320EE66EE66A3DDFE552E552FA
:1015F000060E816EBCDF320EE66EE66A34DFE5521F
:10160000E5521200010E816EB2DF0A0EE66EE66A46
:101610002ADFE552E5521200D9CFE6FFE1CFD9FF2C
:10162000020E816EA4DF0A0EE66EE66A1CDFE5524A
:10163000E552FD0EDBCFE6FFFE0EDB50280DF3502A
:10164000E552E724E76EFE0EE7CFDBFFFD0EDB6A17
:10165000FE0EDB50F36EFD0EDBCFF4FFF350F45CB7
:101660000BE2140E816E83DF320EE66EBFEC10F0DB
:10167000E552FD0EDB2AECD7E552E7CFD9FF120089
:10168000D9CFE6FFE1CFD9FFFE0EDB50816E82DFBE
:10169000320EE66EBFEC10F0E552E552E7CFD9FF0F
:1016A0001200D9CFE6FFE1CFD9FFFD0EDBCFE9FF76
:1016B000FE0EDBCFEAFFEF500EE0FD0EDBCFE9FFC1
:1016C000DB2AFE0EDBCFEAFF01E3DB2AEF50E66EFA
:1016D000D7DFE552EAD7E552E7CFD9FF1200020182
:1016E000046B300E926EF00E936EEF0E006F00C220
:1016F00081FF040E016F0151000821E20051FE0B31
:10170000E842006F00C281FF050EE66EE66AABDEBE
:10171000E552E5528150100B09E08150200B06E0A4
:101720008150400B03E08150800B01E10AD8020197
:10173000040502E1055104D00105016FDCD7CFD7C4
:101740001200F00E936E81CF03F202010315026FB7
:101750000F0E0015006F00510211006F81CF03F2D0
:10176000F00E0315026FF00E025D01E0F7D7936AE9
:1017700006D806C205F20201010E046F1200020132
:10178000076B100E075D14E20751EA6A600FE96EFD
:10179000000EEA22EF50005D08E10751EA6A700F7F
:1017A000E96E000EEA22EFCF06F20729076FE9D7AC
:1017B00006C281FF640EE66EE66A55DEE552E5522A
:1017C00012000201086B070E085D1DE288DF0201AE
:1017D000096F0851EA6A0A0FE96E020EEA2209C28D
:1017E000EFFF0851EA6A0A0FE96E020EEA22EF5093
:1017F000460802E108D004D009C2E6FF41DFE55205
:101800000201082BE0D70851EA6A0A0FE96E020EBE
:10181000EA22EF6A12000201086B070E085D16E269
:101820000851EA6A0A0FE96E020EEA22EF50E66EEC
:1018300027DFE55202010829EA6A0A0FE96E020E63
:10184000EA22EF5001E102D0082BE7D71200D9CFEE
:10185000E6FFE1CFD9FFE652F250800B01E0010E26
:10186000DF6EF29EA69EA69CA684FE0EDB50A96E9D
:10187000FD0EDB50A86E550EA76EAA0EA76EA682AF
:10188000A6B2FED7A694DF50E8B0F28EE8A0F29E92
:10189000E552E552E7CFD9FF1200D9CFE6FFE1CFFD
:1018A000D9FFA69CA69EFE0EDB50A96EA680A8506E
:1018B00000D0E552E7CFD9FF12004D0EE66EE66A82
:1018C0006C0EE66EE5EC0EF0E552E552E5521200C4
:1018D000D9CFE6FFE1CFD9FF040EE126DE6ADE6A4A
:1018E000DE6ADD6ADD52DD52D9CFE9FFDACFEAFFE9
:1018F000D890030EEB50000A08E6400EEE5C0D0E89
:10190000EE58030EEE58000EEE5811E29EAA04D0D7
:1019100028EC10F00ED001D000D0D9CFE9FFDACFFB
:10192000EAFFEE2A000EEE22EE22EE22DDD7000EB6
:1019300000D0146E040EE15C02E2E16AE552E16E51
:101940001450E552E7CFD9FF1200D9CFE6FFE1CF1F
:10195000D9FFE6529EAAFED728EC10F0DF6EDF50CA
:1019600000D0E552E552E7CFD9FF1200D9CFE6FF0C
:10197000E1CFD9FFE6529EAAFED728EC10F0DF6E29
:10198000DFCFE6FF47EC10F0E552DF5000D0E55224
:10199000E552E7CFD9FF1200ABDD8FDFDF0E146E0B
:1019A000200E156E166A14C0E6FF15C0E6FF16C0BD
:1019B000E6FF99EC0EF0E552E552E552DB0E146EAF
:1019C000200E156E166A14C0E6FF15C0E6FF16C09D
:1019D000E6FF99EC0EF0E552E552E552C7DF020151
:1019E000136F520E135D0BE1C1DF0201146F300E55
:1019F000145D01E18090310E145D01E18080540E90
:101A0000135D01E07CD0D10E146E200E156E166AA7
:101A100014C0E6FF15C0E6FF16C0E6FF99EC0EF015
:101A2000E552E552E5520201136B050EE76E1319FC
:101A3000E8AE02D0E73402D0E750135D2CE285DF38
:101A4000E66E13C2E9FFEA6AE9BEEA68150EE92606
:101A5000020EEA22E552E750EF6E13C2E9FFEA6A8E
:101A6000E9BEEA68150EE926020EEA22EF500D08DB
:101A700001E111D013C2E9FFEA6AE9BEEA68150E76
:101A8000E926020EEA22EF50E66E47EC10F0E5522E
:101A90000201132BCAD713C2E9FFEA6AE9BEEA685A
:101AA000150EE926020EEA22EF6A150EE66E020E08
:101AB000E66ED5EC0DF0E552E552F3CF1FF2F4CF10
:101AC00020F21FC2E6FF20C2E6FFC30E146E200EF6
:101AD000156E166A14C0E6FF15C0E6FF16C0E6FFD5
:101AE00099EC0EF0176E050EE15E175080801FC254
:101AF000E6FF20C2E6FF26D8E552E5528090530E5D
:101B00000201135D1DE1FFDCF3CF14F214C214F0E7
:101B1000156A14BE156814C0E6FF15C0E6FFBC0EBA
:101B2000166E200E176E186A16C0E6FF17C0E6FF85
:101B300018C0E6FF99EC0EF0196E050EE15E195023
:101B40002DD71200D9CFE6FFE1CFD9FF020EE12653
:101B5000DE6ADD6ADECF14F0DDCF15F0FD0EDBCFDF
:101B600016F0FE0EDBCF17F015501718E8AE02D0B6
:101B7000173404D01650145C175015580CE2E80EB8
:101B8000E66E030EE66E6FDCE552E552DF2A010ECB
:101B900001E3DB2ADFD7020EE15C02E2E16AE552F3
:0A1BA000E16EE552E7CFD9FF120015
:061BAA00FF0EE3CFEAFF8D
:101BB000E552FF0EE3CFE9FFE552E66AE66AD9CFC8
:101BC000E6FFDACFE6FFFC0EE124D96EFF0EE2203D
:101BD000DA6EE66AE66AE66A200EEF5C06E0090E57
:101BE000EF5C03E0EF6603D03FD0EE50F5D72D0E4B
:101BF000EF5C03E1FF0EE32A03D02B0EEF5C01E163
:101C0000EE502F0EEF6424D03A0EEF6021D0D89022
:101C1000F90EE336FA0EE336FD0EDECFE3FFFE0EDD
:101C2000DDCFE3FFD890F90EE336FA0EE336D89015
:101C3000F90EE336FA0EE336FD0EE350DE26FE0E15
:101C4000E350DD22300EEE5CDE26000EDD22D9D719
:101C5000FF0EE3CFE8FFE85207E0F90EE31EE32AA8
:101C6000FA0ED8B4E306E31EE552E552E552FF0E44
:101C7000E3CFDAFFE552FF0EE3CFD9FFE552E1CF24
:101C8000E9FFE2CFEAFFED52ED52EECFF3FFEFCFE7
:041C9000F4FF12004B
:0C1C94002A0EF66E080EF76E000EF86EB9
:101CA00002010900F550266F0900F550276F03E186
:101CB000266701D03DD00900F550216F0900F5508D
:101CC000226F0900F550236F09000900F550E96EF5
:101CD0000900F550EA6E090009000900F550246F6B
:101CE0000900F550256F09000900F6CF28F2F7CF5B
:101CF00029F2F8CF2AF221C2F6FF22C2F7FF23C24F
:101D0000F8FF0201245302E1255307E00900F550D2
:101D1000EE6E2407F8E22507F9D728C2F6FF29C29C
:101D2000F7FF2AC2F8FF02012607000E275BBFD784
:021D300012009F
:0E1D3200D9CFE6FFDACFE6FFE1CFD9FFE2CF4F
:101D4000DAFFE652E652E652E652D950FB0F146E25
:101D5000FF0EDA20156E14C0DEFFDD6EDECFE6FF6B
:101D6000DDCFE6FFFB0EDBCFE6FFFC0EDBCFE6FFB1
:101D7000FD0EDBCFE6FF2BC2E6FF2CC2E6FF38EC00
:101D800004F0146E070EE15C02E2E16AE552E16ED6
:101D90001450020EF3CFDBFF030EF4CFDBFF020E75
:101DA000DBCF14F0030EDBCF15F014C0F3FF15C02A
:101DB000F4FF040EE15C02E2E16AE552E16EE552F5
:0A1DC000E5CFDAFFE7CFD9FF1200EC
:061DCA00D9CFE6FFDACFDD
:101DD000E6FFE1CFD9FFE2CFDAFFAC6AAB6AFD0ED6
:101DE000DBB0AC88DBA202D0AC8CAB8CDBB4AC8EAD
:101DF000DBA602D0AB8801D0AB8ADBB8AC849E985E
:101E0000DBBAAB86DBAC02D09D8A01D09D9A9E9A4C
:101E1000DBAE02D09D8801D09D98FB0EDB50AF6EEB
:101E2000FB0EFC0EDBCF15F015C014F0156A145034
:101E3000B06EAC8AAB8E949C948EAC50100B04E0C8
:101E4000AC50800B01E1948CE552E5CFDAFFE7CF8F
:041E5000D9FF1200A4
:0C1E5400D9CFE6FFDACFE6FFE1CFD9FFDF
:101E6000E2CFDAFFFB0EDBCF14F0FC0EDBCF15F078
:101E70000001800E15141AE1FB0EDBCFE9FFFC0E0A
:101E8000DBCFEAFFEECFF3FFEDCFF4FFEE2A000E3B
:101E9000EF22F3CFE9FFF4CFEAFFFD0EDBCFEFFF38
:101EA000EF50156AF36E15C0F4FF10D0FB0EDB5037
:101EB000FE0806E1FD0EDBCFE6FFB1EC10F005D029
:101EC000FD0EDBCFE6FFD3EC10F0E552E552E5CF97
:081ED000DAFFE7CFD9FF120091
:081ED80006500B02F3CF02F0EB
:101EE000F4CF03F00C02F3500326000EF420046E2E
:101EF00006500D02F3500426000EF420056E065025
:101F00000E02F350052607500B02F3500326F4503F
:101F10000422000E052207500C02F3500426F45050
:101F2000052207500D02F350052608500B02F3500E
:101F30000426F450052208500C02F35005260950DF
:081F40000B02F350052612000C
:081F4800FE0EE3CFE9FFFF0EDE
:101F5000E3CFEAFFF36AF46AEE5203E0F34AF42AAD
:101F6000FBD71200FF0EE3CFF8FFE552FF0EE3CFE1
:101F7000F7FFE552FF0EE3CFF6FFE552E66AE66AA9
:101F8000E66A0900F55209E0FD0EE32A05E1FE0EBE
:101F9000E32A02E1FF0EE32AF4D7FD0EE3CF07F0B8
:0E1FA000FE0EE3CF08F0FF0EE3CF09F01200B3
:021FAE0009C068
:101FB00013F008C012F008500D02F4CF07F0F3CF71
:101FC00006F009500E02F4CF09F0F3CF08F00D022D
:101FD000F3500726F4500822E86A092212500E0234
:101FE000F3500726F4500822E86A09220EAEFDEFEE
:101FF0000FF01250085E1350095A13AE000C0D502A
:08200000085E0E50095A000CA5
:08200800056A046A036A026A1A
:10201000200EE76ED89006360736083609360236A7
:102020000336043605360B50025C0C5003580D5035
:1020300004580E50055809E30B50025E0C50035A29
:102040000D50045A0E50055A062AE72EE4D7120006
:10205000D9CFE6FFDACFE6FFE1CFD9FFE2CFDAFF53
:10206000E652F20E02012D17ABAC03D02D91ABB0AE
:102070002D81ABB42D85ABB22D87AE50DF6EDF5016
:0E208000E552E552E5CFDAFFE7CFD9FF1200B7
:02208E00D9CFA8
:10209000E6FFDACFE6FFE1CFD9FFE2CFDAFFACAC63
:1020A00004D0AC9002012DB3AC80FD0EDB50AD6EC0
:0C20B000E552E5CFDAFFE7CFD9FF1200C0
:0420BC000D0A533D79
:1020C0002564000D0A257520534547554E444F534E
:1020D000000D0A5449454D504F3D004F4B3E000DF9
:0220E0000A00F4
:0E20E200F36AF46AFF0EE124E96EFF0EE220BD
:1020F000EA6EED6607D02F0EEF6404D03A0EEF6063
:0621000001D0F32A1200D9
:0A210600FF0EE3501B6E480E01D0DF
:102110004C0EE76EE72EFED7E76AE72EFED71B2EA2
:06212000F7D700001200D9
:0A212600000EF36E00EE00F0080E4C
:1021300001D81200EA6002D0EE6AFCD7F350E960E1
:062140001200EE6AFCD75C
:0A21460012EE40F022EE40F0F86ABD
:10215000019C4AEC0EF0D4EC10F0CCEC0CF0FBD768
:0221600012006B
:0E216200FF0EE350ACBA04D0AF6AAB8EAC8A6D
:0E217000949CACA2FED7AD6EF36EF46A120022
:02217E00FF0E52
:10218000E350E84E1200000000D000D000D0E82E4E
:04219000FAD7120068
:0C2194003031323334353637383961626F
:0521A0006364656600A8
:0221A600120025
:0221A800120023
:0221AA00FEFF36
:0421AC00EEEDEBE782
:1021B000DEDDDBD7BEBDBBB77E7D7B773031323312
:0C21C00034353637383941424344454637
:00000001FF
